:1000000048C1000063C1000061C100005FC1000081
:100010005DC100005BC1000059C1000057C1000074
:1000200055C1000053C100000C94201B0C94EC1B24
:100030000C948B164BC1000049C1000047C1000061
:1000400045C1000043C1000041C100003FC10000A4
:100050003DC100000C94041739C1000037C10000F5
:1000600035C1000033C1000031C100002FC10000C4
:100070002DC100002BC1000029C1000027C10000D4
:1000800025C1000023C1000021C100001FC10000E4
:100090001DC100001BC1000019C1000017C10000F4
:1000A00015C1000013C1000011C100002B00140095
:1000B0001A00080015001700E100040016000700F0
:1000C00009000A00E0001D001B00060019000500E1
:1000D000000000000000E3002C00E2002A001300F2
:1000E00012000C0018001C00340033000F000E003A
:1000F0000D000B00280038003700360010001100FA
:10010000E7002C00E600000000000000120353008E
:100110006800720069006D00700034003200000059
:10012000240347007200650065006E004D00610009
:10013000730068006500640050006F007400610087
:1001400074006F0000000403090409023B0002016F
:1001500000A0FA09040000010301010009211101B6
:100160000001224400070581030800010904010081
:10017000010300000009211101000122B60007055A
:1001800082032000011201000200000008EDFE427F
:100190004201000102000105010902A101850209D5
:1001A00001A1000509190129081500250195087507
:1001B0000181020501093009311581257F950275FC
:1001C00008810609381581257F9501750881060586
:1001D0000C0A38021581257F950175088106C0C07B
:1001E00005010980A101850319012AB7001501261F
:1001F000B700950175108100C0050C0901A10185AA
:100200000419012AA002150126A00295017510818A
:1002100000C005010906A1018506050719E029E7C7
:10022000150025019508750181020507190029EFC0
:100230001500250195F075018102050819012905B0
:10024000950575019102950175039101C00501099C
:1002500006A101050719E029E71500250195087594
:100260000181029501750881010507190029FF1513
:100270000026FF009506750881000508190129056B
:1002800015002501950575019102950175039101F0
:10029000C00011241FBECFEFDAE0DEBFCDBF11E0FA
:1002A000A0E0B1E0ECE6FCE302C005900D92AA39B3
:1002B000B107D9F722E0AAE9B1E001C01D92A53B40
:1002C000B207E1F70E94A40F0C94341E99CE81115D
:1002D00012C0683080F4463070F4E42FF0E086E01D
:1002E000689FE00DF11D1124EE0FFF1FE455FF4F35
:1002F00085919491089581E090E00895E8CF089564
:1003000081E00895FDCF0895FBCF0895F9CF0895BA
:10031000F7CF0895FDCF089508950895FDCF08956E
:1003200008950895A6E0B0E0E8E9F1E00C94B01D6E
:1003300049835A839E833091A10189819A81311129
:1003400017C03E81332389F0222379F00AD5182F74
:10035000682F89819A81E4D469817A81812F0E94F2
:10036000DC0C2696E3E00C94CC1DEBD4182FF4CFD4
:10037000F8D469817A81F3CFFC01262F4081518125
:100380006281738184819581CDCFCF93DF93EC011E
:1003900061E0F2DFBE01B6DF882349F061E0CE0103
:1003A000EBDFBE01B1DF8170DF91CF91089580E076
:1003B000FACF0F931F93CF93DF93EC0160E0DCDF64
:1003C0008C01BE01AADFBE01C801A8DFDF91CF9179
:1003D0001F910F9108950F931F93CF93DF93EC011B
:1003E00061E0CADF8C01BE0191DF811106C080E0AF
:1003F000DF91CF911F910F910895BE01C8018ADF4F
:100400008823A9F3BE01C8010E94CE13882379F383
:10041000BE01C8010E94F80F882349F3BE01C8013C
:100420000E94D20F882319F3BE01C8010E94E00D7B
:100430008823E9F2BE01C8010E94F20D8823B9F2B7
:10044000BE01C8010E940B0ED3CF21E030E0A9010C
:1004500002C0440F551F8A95E2F7CA019AC3CF9391
:10046000C82F81E090E00C2E02C0880F991F0A94DB
:10047000E2F70E94E90A8C2FE8DFCF91089581E02E
:100480000895FDCF0895FBCF0895CF93C82F3AD399
:100490008C2FF7DF8C2FF7DFCF91089581E0F5DF08
:1004A0000C942A1780E0F1DF0C943B1739DF0E948F
:1004B000321617C018D035DF0C94361681E0089537
:1004C0000895CF93DF93D82FF9DFC82F882311F039
:1004D0008D2FF6DF8C2FDF91CF9108950895F1CF06
:1004E000089580E0FCCF0E942614F9CFCF930E949C
:1004F0002614C82F80919C018C1771F0C0939C0129
:100500000E94F81660939D0170939E0180939F0155
:100510009093A0018C2FE3DFCF910895ADE0B0E080
:10052000E4E9F2E00C94B11D488759876A877B871C
:100530008C879D87911138D71F8286E0FE013896FF
:10054000DE01119601900D928A95E1F78D8181115E
:100550000CC029813A814B815C816D817E818F81C4
:1005600071D62D96E2E00C94CD1DCE0101960DDFE3
:100570008111EFCFF6CFFC012481213019F4808165
:10058000918120C40895662321F00E9477110C9474
:1005900045120E94C911FBCFCF93882391F0C82F39
:1005A0008CEF8C0F813A78F48C2F0E94D51488231D
:1005B00021F08C2F0E94761582D78C2F0E945F1518
:1005C0007ED7CF91089580E28C0F883040F4C770B9
:1005D00081E001C0880FCA95EAF7C7D6F1CFEBE5F5
:1005E000EC0FE33040F4F0E0E05BFE4F808190E000
:1005F0000E946614E6CFE8E5EC0FEB3150F4F0E032
:10060000EE0FFF1FE65EFE4F808191810E948D14E8
:10061000D8CF83E38C0F8331A0F661E08C2FB3DF5A
:10062000D0CF882351F19CEF980F913A18F40E9493
:10063000761545C790E2980F983048F4877091E09E
:1006400001C0990F8A95EAF7892F95D6F2CF9BE5DD
:10065000980F933020F490E080E00C94661498E5B5
:10066000980F9B3120F490E080E00C948D1493E37C
:10067000980F933110F460E086CF08951F93CF93C5
:10068000DF93182FEB0188DF209731F4812FC9DF2A
:10069000DF91CF911F9108958FE99FE00197F1F7C6
:1006A00000C000002197F0CF70E060E0893311F4C2
:1006B00060E570E0E3CF882311F057D600C70895B6
:1006C000882311F058D6FBC60895B0E0A0E0EBE611
:1006D000F3E00C94AB1D6C01D62FC72FFC011581E4
:1006E000068102950F7037D6E82E8823E9F0E12EB7
:1006F0001123D1F08C2F807F803461F080E28D0F48
:10070000883060F18C2F807E803221F4D23030F13D
:10071000002321F18091930282FF20C082E0F3D672
:100720001AD691E0E82EE926FC2EF2949FE0F922F9
:10073000FBE0FF1508F43CC0EF2DF0E0EE55FC4F58
:100740000C949B1DB003B003E703E703400461046E
:10075000D803D8036504D404E104E104E12CE4CF18
:100760000C2F0F70C07F11F00295007F112381F0D4
:10077000002349F080E28D0F883010F0D11105C0C0
:10078000802FF3D59CD68D2F41C0802FFFD5FACF77
:100790008D2F47DF002361F080E28D0F883010F04D
:1007A000D11103C0802FE7D502C0802FF5D587D6A1
:1007B000EE2009F4B9C0CBD580FDB6C0F601158294
:1007C000C0D518D2C6016FD1BCD522D2ADC02C2F56
:1007D0002F70F22EC07FC03219F0F29480EFF82211
:1007E000DD2341F0D13081F1112309F439C0002318
:1007F000C9F0C9CF8091930282FD10C0112341F04E
:10080000FF2019F08F2DB1D55AD680E0C5DED0CFAC
:1008100080E007DFFF2061F28F2DC5CF112359F053
:10082000011103C08F2D47DFC3CF013009F0C0CFC6
:100830008F2DCED5BDCF0111BBCF8F2D41DF8F2D99
:10084000D2D58F2DB7D5B4CF112321F0063008F0C3
:10085000AFCFE8CF053008F0ABCF8F2D31DFA8CF79
:100860000023D9F3D93349F48FEF97EEE3E08150B9
:100870009040E040E1F700C000008D2FD2DE98CF1D
:100880008C2F86958695837041F0813081F088EFBA
:100890008F0D843008F08CCF44C08D2F9C2F937027
:1008A000111102C080E090E00E94661481CF8D2F6C
:1008B0009C2F9370111102C080E090E00E948D1473
:1008C00077CF612F8D2F5FDE73CF8C2F8370B9F5BB
:1008D000111127C04D2F429546954770440F440F84
:1008E0002D2F2F7030E0042E02C0220F331F0A94E8
:1008F000E2F790E080E0D4FF09C08FE090E002C012
:10090000880F991F4A95E2F780959095822B932B3B
:10091000C695C695C370C23071F078F4C13049F005
:1009200041D10E942614DBDDCDB7DEB7E8E00C94A0
:10093000C71D31D1F6CF3DD1F4CF2BD1F2CF869563
:10094000112311F08C2F8170882359F34D2F42957C
:1009500046954770440F440F2D2F2F7030E0042E22
:1009600002C0220F331F0A94E2F790E080E0D4FF28
:1009700009C08FE090E002C0880F991F4A95E2F706
:1009800080959095822B932BC695C695C370C230E7
:1009900039F040F4C13011F060D1C3CF57D1C1CF8D
:1009A00063D1BFCF13D1BDCFCF70112329F08C2FCE
:1009B00021D18D2F80DEB5CF8D2F82DE8C2F28D1D7
:1009C000B0CFD23F49F168F4D03FC9F0D13F89F0B0
:1009D000112309F441C0002309F43BC08D2FDCDD55
:1009E00056CFD33FF9F0D43F99F78091930282FD1F
:1009F00021C08C2F8F71112399F0FCD048CF112387
:100A000039F0053008F043CF8C2F8F7111D13FCFD3
:100A1000063008F03CCFF8CF8C2F8F71112369F38B
:100A2000F7D035CF112321F08C2F8F71D9D02FCF54
:100A3000D4D02DCF112329F063E08C2F8F714CD5AA
:100A400026CF81E060D5023008F421CF82E05BD56B
:100A50001ECF8C2F8F71D1CF002371F0D93349F481
:100A6000FFEF27EE83E0F15020408040E1F700C027
:100A700000008D2FD6DD0BCF8C2F8F71D1CF0F9330
:100A80001F93CF93DF93EC01688179818D81A3D18E
:100A90008C01F1D07DD0B801CE0117DEDF91CF916E
:100AA0001F910F910895CF93DF93FC01248122239E
:100AB00081F0EC0190DC81110FC04DD4882349F006
:100AC0008D81882331F08091930282FF02C082E001
:100AD0001AD5DF91CF910895CE01D1DFCE0169DC27
:100AE000F8CF90E080E00E94661490E080E00E94E1
:100AF0008D145AD4E4D40E9461120C9445120E94C1
:100B00008D15EFCF40D4FBCF92959F70963089F032
:100B100050F49250923058F4803F19F030F4883EEF
:100B200030F481E008959A50F5CF843FD1F380E00E
:100B30000895883EB0F3813FD1F7F3CFFC012481C3
:100B4000222321F0808191813DD1DECF80E0089584
:100B5000A6E0B0E0EEEAF5E00C94B11D2696E2E0E6
:100B60000C94CD1DA7E0B0E0E8EBF5E00C94B11DCE
:100B70002796E2E00C94CD1D0895FECF0895FDCF99
:100B80000895FADFFCDF9093BD018093BC010895C6
:100B90000895F7CF08952091BC013091BD01822BBB
:100BA000932BEFCF2091BC013091BD018223932381
:100BB000E8CF2091BC013091BD0182279327E1CF7E
:100BC000DBCF0895FDCF0895D7CF0895FDDFFADF7D
:100BD0009093BB018093BA01089590E080E0F6CF36
:100BE00021E030E0A90102C0440F551F8A95E2F7C9
:100BF000CA01ECCF21E030E002C0220F331F8A95FA
:100C0000E2F78091BA019091BB01822B932BDECF4A
:100C100021E030E002C0220F331F8A95E2F72095D1
:100C200030958091BA019091BB0182239323CECF5E
:100C300021E030E002C0220F331F8A95E2F7809155
:100C4000BA019091BB0182279327C0CF2091BA01AE
:100C50003091BB01822B932BB9CF2091BA013091F7
:100C6000BB0182239323B2CF2091BA013091BB0103
:100C700082279327ABCF0895262F277091E001C0DC
:100C8000990F2A95EAF723E0769567952A95E1F77B
:100C9000660F771F660F771FFA01E60FF71F50E008
:100CA00040E0682F70E08191DF0111979B01042ED5
:100CB00002C0369527950A94E2F7217021952827DE
:100CC000292328272C934F5F5F4F4430510559F754
:100CD0000895A82FA77023E0969587952A95E1F7A8
:100CE000880F991F880F991FFB01E80FF91F50E02B
:100CF00040E080E0219130E00A2E02C03695279531
:100D00000A94E2F721703327042E01C0220F0A94BF
:100D1000EAF7822B4F5F5F4F4430510559F7089532
:100D2000282F983068F4863058F4862F622F70E0B0
:100D300026E0929F600D711D112442EA51E09CCF84
:100D40000895983060F4863050F4292F90E062EADC
:100D500071E036E0239F800D911D1124BACF80E011
:100D60000895B0E0A0E0E7EBF6E00C94AA1D7C014A
:100D70000091BA011091BB018091BC019091BD011D
:100D8000082B192BCFE0D0E0CC24C394D12CBC2E5F
:100D9000C6010C2E02C0880F991F0A94E2F7802327
:100DA0009123892B49F4219790F7B12C8B2DCDB746
:100DB000DEB7E9E00C94C61DB7018C2F08D6019769
:100DC00091F3F4CFCF93DF93EC01CBDFBE01FFD5DE
:100DD000DF91CF9108951F93CF93DF93EB01909113
:100DE000A101992331F0CB01EDDFDF91CF911F916C
:100DF0000895882351F0CB01B4DF182F682FCE015E
:100E00008FDFBE01812FE3D5F0CFCB019ADF182F02
:100E1000F8CF1F93CF93DF93C091BE0117E080916D
:100E2000BF018C1304C0DF91CF911F910895D0E0D2
:100E30001C9FF0011D9FF00D1124E054FE4F2081F6
:100E40003181428153816481758186818BDE219657
:100E5000C770E5CF2091F8013091F9014091FA0176
:100E60005091FB016091FC017091FD018091FE01A8
:100E700079CECF93DF938091FE01807F09F04BC044
:100E80008091FD01882309F446C0E091BE01509194
:100E9000BF01C091F901D091F8016091FA01709100
:100EA000FB0147E05E17B9F18E2F90E0E49FF0015F
:100EB0001124E054FE4F2481222381F1489FF00148
:100EC000499FF00D1124DF01A054BE4F11962C91C3
:100ED00011972C1323C02C912D1320C015962C9103
:100EE000159721111BC012962D913C91261B370B93
:100EF000283C310598F48091FE018F7080618093C9
:100F0000FE01EA53FE4F80818F708061808388EFFD
:100F100091E0C9DD7EDFDF91CF910895FC0131962C
:100F2000E770C0CF482F2091BE019091BF0157E0DC
:100F3000291302C080E0089530E0529FF001539FD2
:100F4000F00D1124E054FE4F8181681306C08081AA
:100F5000481303C085818111EECF2F5F3F4F27706B
:100F6000E7CFA4E1B0E0E7EBF7E00C94A71D8C011C
:100F700086E0F801DE011F9601900D928A95E1F757
:100F8000F8018481E58098EFA92E91E0B92E909127
:100F9000FC0191111AC08823A9F0EE2089F0C80144
:100FA000CDDDF82E882361F087E0F801D5010190AE
:100FB0000D928A95E1F7C501DEDA5BDF4BDF59C0A0
:100FC000C80171DDFF24F39454C0C080D1808280B9
:100FD0009380F090FD012091FA013091FB01A40172
:100FE000421B530BFF2009F4E8C0483C510508F0B0
:100FF0009BC0882309F43DC09091F9018091FE01C6
:10100000282F207F09F055C0D91214C09091F80103
:10101000C91210C0E11047C08F7080618093FE013B
:1010200019DF88EF91E03FDD8091FE01F8018683B2
:10103000F12C1FC0E11037C06D2D8C2D73DF6D2D8D
:101040008C2D70DFE82E8111F3CFCF86D88A8F8563
:101050009889B8DE292F22952F70243078F49F705C
:10106000223098F09923A9F0F8019681907F89F4B5
:10107000FE2C8F2D6496ECE00C94C31D2A50223078
:1010800060F0C80110DDEF2CF3CF992311F0882315
:1010900079F3805E8830A8F7EBCF803F48F3815F1B
:1010A000833078F7E5CF8091FE0181608093FE0167
:1010B000BFCFD91212C09091F801C9120EC0E11031
:1010C0000CC08683C801EFDC87E0F801A8EFB1E02F
:1010D00001900D928A95E1F771CFC8012FDD882329
:1010E00009F46ECFEE2009F46BCF8091FE018032BF
:1010F00080F02091F8013091F901398728879B868B
:101100008A869091FC019C871D868E87CE01089669
:10111000CADC87E0F801A8EFB1E001900D928A9552
:10112000E1F7A7DE97DE4ECF9091FE01292F207FB9
:1011300089F4682D9A8A898AA6017A899E2D08DD0C
:1011400088EF91E0B0DC87E0F50111928A95E9F72C
:1011500081DE6ECF882309F48CCF8091F9018D1147
:101160000FC08091F801C8120BC0E11009C096832E
:10117000C80199DC87E0F50111928A95E9F779CFEA
:10118000C801DCDC882309F41BCFEE2009F418CF5A
:101190008091FE01803208F4BCCF2091F80130919B
:1011A000F9013A8329839C828B829091FC019D8373
:1011B0001E828F83CE010196ABCF483C5105A8F526
:1011C000882309F4FFCEFE2CEE2009F4F9CE80919D
:1011D000F9018D111EC08091F801C8121AC08091CA
:1011E000FE0180FD0DC0982F907F51F08683903FC7
:1011F00009F468CF982F907F905F8F70892B61CF13
:1012000087E0F801A8EFB1E001900D928A95E1F72F
:1012100030CFC80193DC81117CCF8091FE018160C9
:101220008093FE01C8013FDC24CF682D9A8A898A09
:10123000A6017A899E2D8CDC87E0F50111928A95B2
:10124000E9F7BCCEAEE0B0E0E8E2F9E00C94B01D06
:10125000288739874A875B876C877D878E87CE0191
:1012600008967FDE882399F16C85662339F02885FE
:1012700039854A855B857D858E8574DC17E0809194
:10128000BE019091BF01891709F457C0819FC00129
:10129000112480549E4F65DE882309F44EC0E091EE
:1012A000BE011E9FF0011124E054FE4F20813181C8
:1012B0004281538164817581868154DC8091BE01B5
:1012C00090E00196877099278093BE01D8CF87E080
:1012D000FE013896DE01119601900D928A95E1F794
:1012E0008C85882359F22091BF0130E0C901019615
:1012F000877099274091BE014817190691F097E031
:10130000929FD001939FB00D1124A054BE4FFE01B7
:10131000319601900D929A95E1F78093BF0179DDA6
:10132000ADCFF0DB1092BF011092BE0187E0E8EF75
:10133000F1E0DF011D928A95E9F72E96E3E00C9427
:10134000CC1D80912702869586958695089580917B
:1013500027028770089590912702977081E009F421
:1013600080E0089580915302089590915302892B53
:10137000809353020895982F90958091530289236A
:10138000809353020895109253020895909152024F
:10139000892B809352020895982F90958091520244
:1013A000892380935202089510925202089508955D
:1013B000FECF089590912802292F282329F08095A7
:1013C000892380932802F4CF08950895FECF0895CD
:1013D00090912902292F2823281721F0982B9093E8
:1013E0002902F4CF089590912902292F282329F06A
:1013F0008095892380932902E9CF0895809129025D
:10140000882321F01092290280E0E0CF0895CF9345
:10141000C091530280915202C82B809129028823E7
:1014200029F0C82B0E94B4148111E8DF8C2FCF91D2
:101430000895CF93DF93C0910201D0910301E7DFBC
:101440008883C0910201D091030148E050E06FE130
:1014500072E0CE010E94EC1D892B59F088E0FE015C
:10146000AFE1B2E001900D928A95E1F7CE010E94C2
:101470003514DF91CF910895CF93DF93C091000190
:10148000D0910101C4DF8983C0910001D091010195
:1014900040E250E06FEF71E0CE010E94EC1D892B1D
:1014A00059F080E2FE01AFEFB1E001900D928A9514
:1014B000E1F7CE010E944214DF91CF9108950E947E
:1014C0001F14882329F08091920287FF01C0D4CF96
:1014D000B0CF0895FECF08959091930292FF0EC071
:1014E00098E0899F90011124622B6093270282DB90
:1014F00080912702869586958695ECCF7BCB1092BE
:10150000270280E0E7CF909127028095892380937E
:101510002702282F277059F4891749F090919302D8
:1015200092FF05C086958695869572DBE8CF089573
:101530009091930292FB222720F9281749F080FB13
:1015400092F99093930282E992E047D082E0DBCF58
:1015500008958091930282FB882780F991E0892782
:10156000E7CF81E0E5CF80E0E3CF60E070E0CB0142
:10157000B9C360E070E0CB01AFD3F7CFA3E0B0E038
:10158000E4ECFAE00C94B11D60D36BD31B82CE0166
:1015900003967ED381E090E09093BD018093BC01DF
:1015A00083D31A8219828A81846080618A83CE0102
:1015B00001968BD3DEDF2396E2E00C94CD1DDECFC7
:1015C000089555C3089542C3089557C3089566C347
:1015D00008956AC308956DC3089577C3089588C3B5
:1015E0000895A6E0B0E0E7EFFAE00C94AF1D0E948A
:1015F000EC168C018091540290915502801791074E
:1016000081F019821A820E94EC16682F49815A8152
:10161000792F80E090E00E948E0210935502009393
:1016200054022696E4E00C94CB1D0E94F8166093B9
:101630005A0270935B0280935C0290935D02609308
:10164000560270935702809358029093590208955E
:1016500008950895FDCF08950895FEDFFBCF089506
:10166000FECF08950895FEDFFBCF8EED9DE07CD484
:10167000F0DFF3CF81E00895FDCF0895FBCF08950B
:10168000089508950895FCDFFCDFFCCF9CDF8111F5
:1016900001C095DF8EE592E098DF82E992E09BDF62
:1016A0007FD495DF76DA8091BA019091BB018ACA26
:1016B0000E94E316C6D3EADF0E941D140E946E0248
:1016C000D2CFA6E0B0E0E7E6FBE00C94A81DD4DFA3
:1016D00081110AC086DF0E941E1415D70E9476026F
:1016E0002696EBE00C94C41DBDD38AE8A82E82E0B8
:1016F000B82E750110E0F70101917F01812F03D30E
:101700001F5F183009F446C00817A9F380915E02E4
:1017100081FDFFD2B3DF982E10E0812FF4D2F82E96
:10172000F50181915F01F81681F100E0EE24E39468
:10173000DF2CD8268D2D8E2109F1CC24C3948F2D3A
:101740008E2109F4C12C9920A1F0602F812F0E94D5
:10175000561681110EC009831A830E94EC16682F59
:101760008B839C8349815A81792F81E09C2D0E9433
:101770008E024C2D602F812F0E946A160F5FEE0C97
:101780000630C1F6F5013197F0821F5F183029F657
:101790004CDFA1CF0813BACF9DCF1F93CF93DF9318
:1017A00018D1EC01C11580E5D807E8F5C11580E432
:1017B000D80708F099C0C03ED10518F5CD3CD10539
:1017C00008F081C0C83AD10570F4C53AD10508F0D7
:1017D00072C0C130D10511F118F0C430D105F0F458
:1017E000D0E0C0E01BC0C33CD105D0F7C85AD0E060
:1017F000CC0FDD1FCD5ADE4F0990D881C02DD464A7
:101800000DC0C11580E2D80708F0C7C0C11581E03E
:10181000D80708F05AC0C83ED10510F7CE01DF91B5
:10182000CF911F910895C03682E5D80718F5C034CE
:1018300082E5D80708F066C0C03282E5D80708F014
:101840005AC0C11582E5D80708F48FC02C2F269501
:10185000269580E2289F900111248C2F8370C1E08F
:10186000D0E002C0CC0FDD1F8A95E2F7C22BD32B4C
:10187000DD68D4CFC03A82E5D80760F4C03882E58D
:10188000D80708F454C0CF71D0E0DC2FCC27C46F48
:10189000D06AC4CFC03C82E5D80708F45BC0C03E24
:1018A00082E5D80708F09CCFDC2FCC27CC27DF714E
:1018B000C06FD06AB3CFC55AD0E0C757DE4FC881DA
:1018C000D0E0D064ABCFD065A9CF8D2F26D1182F13
:1018D000CE0199277ED0C12FD0E0DC2FCC27CC279A
:1018E000DF71C82BD92B9ACFCE01992772D0CC2784
:1018F000DF70D06AF6CFCF71D0E0DC2FCC27C16F7C
:10190000D06A8CCF2C2F26952695277080E2289FB1
:10191000900111248C2F8370C1E0D0E002C0CC0F65
:10192000DD1F8A95E2F7DC68C22BD32B77CF2C2FF3
:1019300026952695277080E2289F900111248C2FF0
:101940008370C1E0D0E002C0CC0FDD1F8A95E2F7C2
:10195000DA68EACF8C2F8F71E0D0C82FD0E0DC2F6F
:10196000CC27CC27DF71D06259CF8C2F8F71D5D087
:1019700055E0D695C7955A95E1F7CF70D0E0DC2FAA
:10198000CC27282F30E084FF06C044E0220F331F0D
:101990004A95E1F73327D069C7CF8D2F8F71BDD01E
:1019A000182FCE01992715D0C12FD0E0DC2FCC27DE
:1019B000CC27DF71906295CF783030F4663020F418
:1019C000462F672F0C947E0190E080E00895F4DFAD
:1019D000E4CE82389105B9F1B0F48133910509F470
:1019E0007DC048F48932910509F46DC08A329105B1
:1019F00009F479C008958533910509F45FC08933EE
:101A0000910509F10895833E9105D9F138F4803E9E
:101A1000910529F1823E910579F10895863E91055F
:101A2000D9F1873E910509F43EC0843E910541F508
:101A30002091930221FF24C08091920284FD19C05D
:101A400087EE90E0089520919202237009F056C02D
:101A50002091930223FF14C089E290E00895209121
:101A6000920220FD38C03091930230FF09C024FF5C
:101A70003FC090E080E008952091920222FDF7CFD0
:101A800008952091920222FD36C03091930230FDDC
:101A900035C024FDEECFF4CF2091920223FFF0CF8A
:101AA00024FDE7CFCDCF2091920223FD2AC03091B3
:101AB000930231FFEECF84EE90E0089520919202E0
:101AC00025FDCACF08952091920225FD1DC02091C9
:101AD000930223FFD5CF89E390E0089520919202ED
:101AE00026FD15C008952091920226FD13C0089589
:101AF00083EE90E0089582EE90E0089580EE90E00D
:101B0000089586EE90E0089585E390E008958AE2D6
:101B100090E0089581E390E0B3CF9091920292FF1C
:101B200010C041E0282F2471243009F040E031E05A
:101B3000282F2871283009F030E0431711F02CE0ED
:101B4000822793FF10C041E0282F2471243109F02F
:101B500040E031E0282F2871283109F030E04317A8
:101B600011F02CE082273091930230FF10C051E039
:101B7000282F2171213009F050E041E0282F2871F1
:101B8000283009F040E0541711F029E0822731FF96
:101B900010C041E0282F2171213109F040E031E0EF
:101BA000282F2871283109F030E0431711F029E07F
:101BB000822794FF02C083FD877E089580E0089508
:101BC000CF939C01205E3245C1E02032310538F4CC
:101BD000FB01C581C11103C08F710E942F028C2FA0
:101BE000CF9108959C01FB018581882391F02B35CD
:101BF000FCE73F0761F02C359CE7390729F02A35CF
:101C00003C4741F4AEDC01C0A4DC80E00895ABDCCD
:101C1000FCCF81E008959C01FB018581882399F028
:101C20002130FCE73F0761F023309CE7390739F0AA
:101C300021153C4749F40E944E0280E00895C1DC22
:101C40000E945202FACF81E00895089590E080E06A
:101C50000E94011E21E0833E9E4F09F020E0822F6A
:101C6000089563EE7EEF90E080E00C94201E6FEF0D
:101C70007FEF90E080E00C94201ECF93DF93EC0187
:101C800082E090E00E94F91D8883DF91CF91089552
:101C9000FC01608182E090E00C94061E83E090E0FD
:101CA0000E94F91D90E00895682F83E090E00C9465
:101CB000061ECF93DF93EC0184E090E00E94011EAA
:101CC00099838883DF91CF910895FC0160817181B0
:101CD00084E090E00C94201EAB01BC018FE090E00A
:101CE0000C94181EAB01BC0183E190E00C94181E0B
:101CF000682F8EE090E00C94061E0895FECF0895A4
:101D00000895FECF0895E82FF0E0E456FD4F80815E
:101D10000895089580EA8A95F1F7089500C008951E
:101D2000F9CF0895F894E82FE295EF70F0E031A133
:101D3000282F2F7081E090E001C0880F2A95EAF7E4
:101D4000982F9095932391A392A1892B82A37894A5
:101D500008950F931F93CF93DF93C2E9D1E0899148
:101D60008F3F09F0DFDF81E0CA39D807C1F7CCE83F
:101D7000D1E002E911E089918F3F09F0D3DF0C1720
:101D80001D07C9F7DF91CF911F910F910895B0E022
:101D9000A0E0EDECFEE00C94AB1DEC01062F10E092
:101DA000C8018E569E4F7C01FC0190819F3F09F433
:101DB00041C0D62EF894E92FE295EF70F0E081A1B2
:101DC0009F7021E030E001C0220F9A95EAF7822B44
:101DD00081A382A12095282322A378949FDFECE899
:101DE000F1E031E0C12C21912F3F49F1A22FA295C2
:101DF000AF70B0E090968C9190E02F7002C09595F6
:101E000087952A95E2F780FD1AC0832FC82A330FE1
:101E100081E0E239F80739F7F70180818F3F09F057
:101E200081DF61E0C11001C060E08D2D79DFC00F5E
:101E3000D11FC882CDB7DEB7E8E00C94C71D80E0A3
:101E4000E5CF87DF88E0ECE9F2E0DF01982F1D9213
:101E50009A95E9F7E4E9F2E0DF011D928A95E9F746
:101E600038D04CCFA8E0B0E0E8E3FFE00C94AE1D22
:101E70008E010F5F1F4F88E0F80111928A95E9F7F4
:101E8000F12C6F2DC80183DFF394F8E0FF12F9CF36
:101E900048E050E0B80184E992E00E94EC1D41E086
:101EA000009709F440E0892B41F088E0F801A4E9AB
:101EB000B2E001900D928A95E1F76CE972E084E955
:101EC00092E008D0182F1DDF812F2896E5E00C94B2
:101ED000CA1D0895EF92FF920F931F93CF93DF9344
:101EE0007C018B01C42F442371F081E08093610257
:101EF00073D79093600280935F0280E0CDB7DEB726
:101F0000E6E00C94C91DD0916102DD23B1F380910C
:101F10005F0290916002EFD6059778F348E050E0B9
:101F2000B701C8010E94EC1D892B41F088E0F70140
:101F3000D80101900D928A95E1F7CD2F10926102A0
:101F40008C2FDCCFBECB0895DFD60E9471188DDBBD
:101F50000E948918ADDB0E9492180E949518F2DF4A
:101F60000E94AB1890DBF9CF90939B0180939A016C
:101F7000089527CB089580E0C6DE8170089572DF52
:101F80002FEF86E791E0215080409040E1F700C0BC
:101F9000000068DFF0DF882311F0EBDF5BC70895F6
:101FA000EECF0895CF93DF9386319C47F9F4EB0190
:101FB000D9D99D81992389F08A7A91E009F490E03A
:101FC00090936202811107C089E279D578DA80E0C6
:101FD000DF91CF91089585E3F8CF8091620281115E
:101FE00003C089E283D5F2CF85E3FCCF81E0F0CF57
:101FF000CF93DF93EC01FB018581882309F4EEC0C8
:102000009E0130572332310508F0CEC082E992E0BC
:10201000E2DAFE01E150F047E232F10508F026C0B5
:10202000EC5EFF4E0C949B1D7010E0107810421077
:1020300046107C104A1080108C105610D9105A107F
:1020400090105E109410BC1062109810C3106810AD
:102050009E10A6104E108410521088106C10A21002
:10206000B210CC10D7103C107410E710809192027F
:1020700081608093920292C08091930288608093E5
:1020800093028CC0809192028260F3CF8091920281
:102090008460EFCF809192028860EBCF80919302B1
:1020A0008160EDCF809193028260E9CF80919202AE
:1020B0008061DFCF809192028062DBCF80919202BB
:1020C0008064D7CF0E948205809192028068D1CF30
:1020D000809192028860DCCF809193028260E0CF91
:1020E000809192028E7FC5CF80919302877FC7CF68
:1020F000809192028D7FBDCF809192028B7FB9CF6C
:1021000080919202877FB5CF809193028E7FB7CF67
:10211000809193028D7FB3CF809192028F7EA9CF61
:10212000809192028F7DA5CF809192028F7BA1CF6B
:102130000E948205809192028F779BCF80919202BC
:10214000877FDCCF809193028D7FE0CF80919202D8
:1021500082FB992790F921E0922790FB82F990FB6E
:1021600083F987CF80919302982F909591708E7FFD
:10217000892B90FB81F983CF90919202892F8F7BDD
:1021800096FF806476CF0E94820590919202892FFB
:1021900097FB87F980586DCF81E021DA82E992E0E0
:1021A0001CDA0E94820580E0DF91CF91089580E0E3
:1021B000F4CF90919202892F8F7E94FF806159CF46
:1021C00090919202892F8E7F90FF816052CF9091E3
:1021D0009302892F877F93FF886051CF81E0E4CFFE
:1021E000282F35EB2303C001112497FF04C080582A
:1021F0009109892F089580589F4FFBCF80916902E4
:1022000080FF0DC06091090170E0660F771F603894
:10221000710580F56115710579F1862F089581FFAB
:1022200007C06091090184E0689FB0011124EFCFDD
:1022300082FF04C06091090188E0F6CF2091680216
:102240002223A9F0909108016091090188E0689F1C
:10225000B00111242917D8F6269FA001279F500D01
:102260001124692F70E0CA010E94881DD0CF68E058
:1022700070E0D3CF8FE7089581E0089580916902DF
:1022800080FF0CC06091050170E0759567957595AC
:1022900067956115710549F1862F089581FF06C084
:1022A0006091050170E075956795F3CF6091050128
:1022B00082FD0BC0909167029923A1F06091040107
:1022C00080910501961738F0682F70E0603871052D
:1022D00000F38FE70895899FC001112470E00E94E8
:1022E000881DF4CF61E070E0D7CF81E008958D3C88
:1022F00029F484DF819580936D0208958E3C11F45A
:102300007DDFF9CF8F3C29F479DF819580936C02D2
:102310000895803D11F472DFF9CF893D21F4AEDFDD
:1023200080936E0208958A3D19F4A8DF8195F8CF55
:102330008B3D29F4A3DF819580936F0208958C3D36
:1023400011F49CDFF9CF9FE2980F983070F4815D13
:10235000990B21E030E001C0220F8A95EAF78091C5
:102360006B02822B80936B0208958D3D31F4809136
:10237000690281608093690208958E3D21F4809105
:1023800069028260F7CF8F3DB9F78091690284605E
:10239000F1CF8D3CD9F490916D0297FF1DC0109242
:1023A0006D0280916C02811106C080916D028111D5
:1023B00002C01092680280916E02811106C0809165
:1023C0006F02811102C01092670208958E3CD9F409
:1023D00090916D0219161CF39FE2980F983008F047
:1023E0003FC0815D990B21E030E0A90102C0440F9C
:1023F000551F8A95E2F7CA01809590916B02892357
:1024000080936B02CECF90916C028F3C29F497FFA2
:10241000E3CF10926C02C5CF803D19F41916CCF3AE
:10242000DBCF90916E02893D29F41916ACF610921B
:102430006E02B7CF8A3D19F497FFCECFF8CF8B3D10
:1024400039F490916F0297FFC7CF10926F02A9CF16
:102450008C3D09F0C1CF90916F021916B4F3BCCF37
:102460008D3D31F4809169028E7F8093690299CF0E
:102470008E3D21F4809169028D7FF7CF8F3D09F069
:1024800090CF809169028B7FF0CFA6D420916C020F
:10249000211104C020916D02222321F09093660245
:1024A0008093650220916E02211104C020916F0279
:1024B000222321F090936402809363028AE692E0E3
:1024C000F3C186E0EAE6F2E0DF011D928A95E9F7C2
:1024D0001092680210926702109269020895FC013E
:1024E000828181110EC0838181110BC08481811191
:1024F00008C091E08581811101C090E0892F817031
:10250000089581E0FCCFA6E0B0E0E9E8F2E10C94A8
:10251000B01D86E0EAE6F2E0DE01119601900D9230
:102520008A95E1F710926C0210926D0210926E0281
:1025300010926F028B81811103C08C81882381F0FE
:102540008091650290916602D6D3AC0190916802A9
:102550009923B9F180910A018417150608F43EC049
:102560008D81811103C08E81882389F0809163025F
:1025700090916402C0D3AC0190916702992309F451
:1025800063C0809106018417150608F46BC0BE0174
:102590006F5F7F4F8AE692E0D9D2811104C08AE64C
:1025A00092E09DDF811171DF86E0FE013196AAE69F
:1025B000B2E001900D928A95E1F72696E3E00C9443
:1025C000CC1D20910B018AE0289F90011124241733
:1025D000350730F69F5F9093680202C09F3FD1F7A6
:1025E0001B81112351F00ADE9FEF11160CF491E0CC
:1025F000899F802D112480936C021C81112351F03E
:10260000FDDD9FEF11160CF491E0899F802D1124C0
:1026100080936D0280916C02882309F4A1CF109100
:102620006D02112309F49CCFDBDD882349F08093F0
:102630006C02812FD5DD882329F080936D0290CF25
:1026400081E0F5CF81E0F9CF209107018AE0289F52
:10265000900111242417350708F099CF9F5F9093BC
:10266000670202C09F3FD1F71D81112351F006DEA2
:102670009FEF11160CF491E0899F802D1124809317
:102680006E021E81112351F0F9DD9FEF11160CF43B
:1026900091E0899F802D112480936F0280916E02BA
:1026A000882309F474CF10916F02112309F46FCFBE
:1026B00097DD882349F080936E02812F91DD882376
:1026C00029F080936F0263CF81E0F5CF81E0F9CFED
:1026D0000F931F93CF93DF93C42FD22FFC018581DB
:1026E0008823C1F04093720277D390937102809354
:1026F000700280E28C0F883040F4C77081E001C026
:10270000880FCA95EAF70E945B03DF91CF911F9172
:102710000F91089510917202141331C080917002CC
:1027200090917102E8D2883C910548F5C0E2CD0F46
:102730001D17B9F080E2810F883040F4177081E0F6
:1027400001C0880F1A95EAF70E946003C83010F59F
:1027500081E09D2F977001C0880F9A95EAF70E943B
:102760005B03802F0E945403C83078F6D77081E055
:1027700001C0880FDA95EAF70E946003C6CF80E2B5
:102780008C0F883010F6C77081E001C0880FCA95A1
:10279000EAF7F2CF802F0E945403B7CF0F93FC01CA
:1027A000E851FC47E730F10508F039C0CB01E552AC
:1027B000FC4E0C949B1DF113F713E213EB13FD1366
:1027C0000314091406E221EE41EE6AE17CE780DFA2
:1027D00080E00F91089507E225EE45EE6BE17CE77E
:1027E000F6CF06E221EE40EE68E17CE7F0CF07E2AB
:1027F00025EE44EE69E17CE7EACF06E221EE42EE07
:102800006CE17CE7E4CF07E225EE46EE6DE17CE784
:10281000DECF08E221E045EE6EE17CE7D8CFFB0198
:102820008581882319F010927202D3CF81E0D1CF35
:102830009093780280937702089508950895F1D1D6
:1028400091E0813009F090E0892F0895E0917702BE
:10285000F0917802309739F00190F081E02D3097B7
:1028600011F00995089580E00895E0917702F091C4
:102870007802309731F00280F381E02D309709F033
:1028800009950895E0917702F0917802309759F018
:1028900024813581232B39F026E0DC012C93048040
:1028A000F581E02D09950895E0917702F091780285
:1028B000309759F026813781232B39F022E0DC0153
:1028C0002C930680F781E02D09950895A3E0B0E0F0
:1028D000ECE6F4E10C94B11D209175023091760282
:1028E00028173907B1F09093760280937502E09132
:1028F0007702F0917802309761F00084F185E02D45
:10290000309739F023E029839B838A83CE01019697
:1029100009952396E2E00C94CD1DA3E0B0E0E3E935
:10292000F4E10C94B11D20917302309174022817C8
:102930003907B1F09093740280937302E0917702AB
:10294000F0917802309761F00084F185E02D3097A6
:1029500039F024E029839B838A83CE01019609956F
:102960002396E2E00C94CD1DCF93DF93C09102013A
:10297000D0910301229663DF882381F08091920237
:1029800087FF0CC0C0910001D091010122969EE109
:1029900080E0915028F4DF91CF91089596E0F8CF30
:1029A00029912223B1F38F5FF4CFCF93882321F1B4
:1029B000C82F45DF882319F18091920287FF1FC03D
:1029C000EC2FE695E695E695EE31B0F480910001A6
:1029D00090910101E80FF92FF11D228130E0C770BD
:1029E00081E090E002C0880F991FCA95E2F7282382
:1029F000392381E0232B09F480E0CF910895809161
:102A0000020190910301FC013296089621912C1746
:102A100021F0E817F907D1F7EFCF81E0EECF9C0165
:102A2000FC0132969FEF80E04191461751F09F3FA5
:102A300019F4411101C0982F8F5F8630A9F79F3F8D
:102A400009F40895290F311D97FD3A95F901628324
:102A50000895FC01329608962191261303C0DF01E8
:102A600011971C92E817F907B9F70895E62FE69534
:102A7000E695E695EE3168F4E80FF92FF11D6770E1
:102A800021E030E001C0220F6A95EAF78281822BB3
:102A900082830895E62FE695E695E695EE3170F48B
:102AA000E80FF92FF11D677021E030E001C0220F1F
:102AB0006A95EAF720958281282322830895CF938F
:102AC000C82FBDDE6C2F882359F08091920287FFBA
:102AD00007C08091000190910101C8DFCF91089556
:102AE00080910201909103019ADFF8CFCF93C82F14
:102AF000A6DE6C2F882359F08091920287FF07C0D1
:102B00008091000190910101C5DFCF9108958091DE
:102B10000201909103019DDFF8CF91DE882379F0C7
:102B20008091920287FF0BC0E0910001F0910101BA
:102B300032968EE1DF011D928A95E9F70895E091C2
:102B40000201F0910301329686E0F4CFDC01FB0133
:102B500011969C9111978181981322C012968C91A5
:102B60001297882319F0928189131AC013968C91B9
:102B70001397882319F09381891312C015968C91AD
:102B80001597882319F0958189130AC014969C9192
:102B9000992321F081E02481291303C080E001C042
:102BA00081E0817008950895FECF089581110CC0D1
:102BB00081E080930F0160910C0170910D01809173
:102BC0000E0190910F01F0CF82E0F3CF83E080936C
:102BD0000F0160910C0170910D0180910E01909197
:102BE0000F01E2CFE3CF089581E080930F01609160
:102BF0000C0170910D0180910E0190910F01D4CFC5
:102C0000F3CF089591E0811101C090E090930E01FF
:102C100060910C0170910D0180910E0190910F0156
:102C2000C3CF80910E01089580930D0160910C0136
:102C300070910D0180910E0190910F01B5CF80919F
:102C40000D01089580930C0160910C0170910D01AC
:102C500080910E0190910F01A7CF80910C010895F2
:102C600008950895FECF089508950895F9CF089521
:102C70000F931F93CF93DF93F7DFF4D8F6DF09E7C5
:102C800012E0C0E0D0E08C2F3ED8F80181938F0194
:102C900091E0811101C090E0D92BCF5FC83099F746
:102CA0008D2FDF91CF911F910F910895E82FF0E0C4
:102CB000E758FD4F208130E081E090E002C0880FAE
:102CC000991F6A95E2F72823392381E0232B09F421
:102CD00080E0089541110EC0E82FF0E0E758FD4F65
:102CE00021E030E001C0220F6A95EAF7209580814B
:102CF000282320830895CF93DF93EC016DD08C1BA4
:102D00009D0BDF91CF91089585B7806885BF85B70A
:102D1000806885BF08951F920F920FB60F921124FD
:102D20008F939F93AF93BF9380918102811113C0C2
:102D30008091A4029091A502A091A602B091A70251
:102D40004196A11DB11D8093A4029093A502A0936A
:102D5000A602B093A702BF91AF919F918F910F9060
:102D60000FBE0F901F9018958091AC02843031F106
:102D70000E9456021092810288E190E020E40FB692
:102D8000F894A895809360000FBE2093600083B7ED
:102D9000817F846083BF83B7816083BF7894889587
:102DA00083B78E7F83BF0FB6F894A895809160009B
:102DB000886180936000109260000FBE08950E94A9
:102DC00082050C945A0282E084BD93E095BD9AEF8F
:102DD00097BD80936E0008952FB7F8948091A40258
:102DE0009091A502A091A602B091A7022FBF0895CD
:102DF0002FB7F8946091A4027091A5028091A60269
:102E00009091A7022FBF089578941F920F920FB64A
:102E10000F9211248F939F93AF93BF938091A4023D
:102E20009091A502A091A602B091A7020196A11DC2
:102E3000B11D8093A4029093A502A093A602B09323
:102E4000A702BF91AF919F918F910F900FBE0F90EE
:102E50001F90189587E797E79093010880930008E3
:102E600088E19AE00FB6F894A895809360000FBEB1
:102E700090936000FFCF88E19AE00FB6F894A89590
:102E8000809360000FBE90936000FFCF9B019091F4
:102E9000AC029430E9F48F708093E9008FEF909149
:102EA000E800815095FD06C095ED9A95F1F7000078
:102EB0008111F5CF8091E80085FF0AC0BA01C901F0
:102EC00050E040E0BAD18091E8008E778093E8002E
:102ED000089543E050E0BC0182E0D8CF46E050E0E6
:102EE000BC0182E0D3CF40E250E0BC0182E0CECF13
:102EF000CF93DF93EC0195DE48E050E0BE0181E026
:102F0000C5DF88E0FE01A2E8B2E001900D928A954B
:102F1000E1F7DF91CF9108958091AB02811107C055
:102F20001AD371D38091E20084608093E200089507
:102F30001092AB02089558DE81E064CE6091A80241
:102F400081E0611101C080E041CE9091AC0281E04E
:102F5000943009F080E06091A80244CE42E061EC38
:102F600081E077D242E261EC82E073D29091AC02D0
:102F700081E0943009F080E06091A80217CE809142
:102F8000AE02833009F461C030F48130D9F182306F
:102F900009F497C008958A3009F486C08B3009F48B
:102FA0006EC0893009F050C08091AD02813209F0C5
:102FB0004BC08091B1029091B202029708F044C0D8
:102FC0008091E800877F8093E8008091E80082FF8D
:102FD00037C08091F3009091F200892798278927C4
:102FE000029731F48091F100813011F0863019F4AC
:102FF0008091F10019DE8091E8008B778093E800E2
:103000005CD222C08091AD02813AF1F48091E80057
:10301000877F8093E8008091B1029091B202892B62
:1030200059F468E082E892E070E054D18091E800C1
:103030008B778093E800089560E090E080E0F4CF23
:103040008091AC028111C1CF08958091AD02813A87
:10305000D9F78091B1029091B202892BA9F78091A2
:10306000E800877F8093E8008091E80080FFFCCF34
:10307000D8DD8093F1008091E8008E77BFCF8091FA
:10308000AD02813209F78091B1029091B202892B91
:10309000D9F68091E800877F8093E8000ED2809176
:1030A000AF02B0DD0C9482058091AD02813261F6F1
:1030B0008091E800877F8093E800FFD18091B00283
:1030C000C1CD8091AD02813A09F0BECF8091E80078
:1030D000877F8093E8008091E80080FFFCCFBDDD12
:1030E000C8CF84B7877F84BF0FB6F894A895809126
:1030F0006000886180936000109260000FBE80E8DD
:1031000090E00FB6F89480936100909361000FBE39
:1031100077CD21D278D2E2EEF0E0808184608083A6
:103120007894DBC480E191E083CB8091AC02853060
:1031300029F48091AC02853011F041CE089514DE5F
:1031400097DD8823B1F38091AA02882391F35FD0A1
:103150000E948205EECF08959A014091B3025091EA
:10316000B40200C0492F55274330510571F158F47E
:1031700041305105E9F04230510511F190E080E015
:1031800050E040E019C04132510591F14232510501
:10319000A9F784E490E04DE452E06115710561F017
:1031A00086EB90E047E951E06130710529F0E6CF08
:1031B00082E190E045E851E0F901518340830895B0
:1031C0008BE390E04AE451E0F7CF992781309105F5
:1031D00061F028F0029791F6ECE0F1E002C0E6E43D
:1031E000F1E0849190E0AF01E7CFE0E2F1E0F9CFC8
:1031F00089E090E04CE551E061157105E9F289E064
:1032000090E045E751E061307105B1F2B7CF80E160
:1032100089BD82E189BD09B400FEFDCF8091D8004F
:103220008F7D8093D8008091E00082608093E000E1
:103230008091E00081FDFCCF0895AF92BF92CF92C4
:10324000DF92FF920F931F93CF93DF936C01EB01FB
:103250008A0152D1F82E811123C00115110539F0D0
:10326000F80180819181C81BD90BC80ED91EB12CE1
:10327000A12C2097A9F08091E80085FD21C08091C4
:10328000E8008E778093E80001151105A1F0F801A0
:1032900080819181A80EB91EB182A08285E0F82EAE
:1032A0008F2DDF91CF911F910F91FF90DF90CF90E5
:1032B000BF90AF90089520D18823D9F2F82EF0CF97
:1032C000F60181916F018093F1002197FFEFAF1A12
:1032D000BF0ACFCFFC018091B3029091B402861750
:1032E0009707A0F06115710529F49091E8009E7789
:1032F0009093E80090E06115710551F4911108C0B8
:103300008091E80082FF35C080E00895BC01F2CFD3
:103310008091AC028823C9F18530C9F18091E80021
:1033200083FD31C08091E80082FDEACF8091E80002
:1033300080FFE1CF2091F3008091F200322F282FFF
:103340006115710519F02830310558F091E02830E9
:10335000310509F090E02091E8002E772093E800F5
:10336000CACF81918093F100615071092F5F3F4F67
:10337000E7CF8091AC02882341F0853041F0809105
:10338000E80083FFBDCF81E0089582E0089583E0E7
:103390000895FC018091B3029091B40286179707BB
:1033A000A0F06115710529F48091E8008E77809373
:1033B000E80090E06115710551F4911108C0809109
:1033C000E80082FF36C080E00895BC01F2CF809112
:1033D000AC028823D1F18530D1F18091E80083FDE2
:1033E00032C08091E80082FDEACF8091E80080FF42
:1033F000E1CF2091F3008091F200322F282F611548
:10340000710519F02830310558F091E02830310568
:1034100009F090E08091E8008E778093E800CACFB1
:1034200084918093F1003196615071092F5F3F4F75
:10343000E6CF8091AC02882341F0853041F0809145
:10344000E80083FFBCCF81E0089582E0089583E027
:103450000895982F973028F08F708093E90081E0CD
:1034600008959093E900242F762F50E0981731F0BB
:103470007091EC002091ED005091F00021FD02C010
:103480009F5FE8CF3091EB003E7F3093EB003091AF
:10349000ED003D7F3093ED003091EB0031603093D3
:1034A000EB007093EC002093ED005093F00020911E
:1034B000EE0027FDE5CF80E008958091AD0287FF03
:1034C00013C08091E80082FF06C08091E8008B77EE
:1034D0008093E80004C08091AC028111F2CF08957E
:1034E0008091AC028823D9F38091E80080FFF8CF67
:1034F0008091E8008E77ECCF2091E4003091E500D8
:1035000085E69091EC0090FF06C09091E80090FF56
:1035100006C080E008959091E80092FDFACF909166
:10352000AC02992391F0953091F09091EB0095FDCC
:1035300010C04091E4005091E5002417350709F3CD
:1035400081509A01F1F684E0089582E0089583E0C5
:10355000089581E0089567D06ED0E0EEF0E08081BC
:1035600081608083E8EDF0E080818F77808319BCF3
:10357000A7EDB0E08C918E7F8C9380818F7E8083CD
:103580001092AB0208950F931F93CF93DF934BD00C
:1035900052D0C8EDD0E088818F7788838881806899
:1035A000888388818F7D888319BC1092AC02109229
:1035B000A8021092AA021092A90200EE10E0F801EF
:1035C00080818B7F808388818160888342E060E096
:1035D00080E03FDFE1EEF0E080818E7F8083E2EEED
:1035E000F0E0808181608083808188608083F80141
:1035F00080818E7F8083888180618883DF91CF91F5
:103600001F910F910895E8EDF0E080818F7E808317
:10361000E7EDF0E080818160808384E082BF81E01B
:103620008093AB02B0CFE8EDF0E080818E7F8083A5
:103630001092E20008951092DA001092E1000895CD
:103640001F920F920FB60F9211242F933F934F9317
:103650005F936F937F938F939F93AF93BF93EF93FA
:10366000FF938091E10082FF0AC08091E20082FF17
:1036700006C08091E1008B7F8093E1002DD2809184
:10368000DA0080FF18C08091D80080FF14C08091BC
:10369000DA008E7F8093DA008091D90080FF8FC09E
:1036A00080E189BD82E189BD09B400FEFDCF81E0E2
:1036B0008093AC0231DC8091E10080FF18C08091E2
:1036C000E20080FF14C08091E2008E7F8093E200D0
:1036D0008091E20080618093E2008091D800806256
:1036E0008093D80019BC85E08093AC0227DC8091E0
:1036F000E10084FF28C08091E20084FF24C080E1C3
:1037000089BD82E189BD09B400FEFDCF8091D8005A
:103710008F7D8093D8008091E1008F7E8093E100BF
:103720008091E2008F7E8093E2008091E2008160D0
:103730008093E2008091A802882309F445C084E0C8
:103740008093AC0202DC8091E10083FF27C080916E
:10375000E20083FF23C08091E100877F8093E10036
:1037600082E08093AC021092A8028091E1008E7FEB
:103770008093E1008091E2008E7F8093E20080914F
:10378000E20080618093E20042E060E080E061DE80
:103790008091F00088608093F000CDDBFF91EF9185
:1037A000BF91AF919F918F917F916F915F914F9159
:1037B0003F912F910F900FBE0F901F90189519BC3D
:1037C0001092AC02B5DB77CF8091E30087FD02C099
:1037D00081E0B6CF83E0B4CF1F920F920FB60F9265
:1037E00011242F933F934F935F936F937F938F9306
:1037F0009F93AF93BF93CF93EF93FF93C091E90053
:10380000CF708091EC001092E9008091F000877FEA
:103810008093F00078941BD01092E9008091F00022
:1038200088608093F000C093E900FF91EF91CF9101
:10383000BF91AF919F918F917F916F915F914F91C8
:103840003F912F910F900FBE0F901F901895AAE2F5
:10385000B0E0ECE2FCE184C1EDEAF2E08091F1003D
:10386000819322E0E53BF207C9F789DB8091E8000C
:1038700083FF43C08091AD029091AE029A3008F070
:103880003CC0E92FF0E0EA5BF34E55C1501C761CBA
:103890007D1C761C7D1CCC1CED1C7D1C411D4E1D11
:1038A000803889F0823849F58091B1028F70873075
:1038B00020F58093E9008091EB0085FB882780F953
:1038C0001092E90006C08091A9029091AA0291117C
:1038D00082609091E800977F9093E8008093F100D8
:1038E0001092F1008091E8008E7726C0282F2D7F5E
:1038F00021F4882399F0823019F18091E80083FF48
:103900000AC08091E800877F8093E8008091EB00F7
:1039100080628093EB00AA96E3E03EC18091AF0203
:10392000813059F7933009F080E08093AA02109219
:10393000E9008091E800877F8093E800BEDDDDCF5D
:103940008091AF028111F3CF8091B1028F702FEF80
:10395000280F263090F68093E9002091EB0020FF9D
:10396000E6CF933031F48091EB0080628093EB00DE
:10397000DECF9091EB0090619093EB0021E030E07E
:1039800001C0220F8A95EAF72093EA001092EA001C
:103990008091EB008860EACF8111AFCF1091AF0228
:1039A0001F778091E3008078812B8093E3008091E2
:1039B000E800877F8093E80080DD8091E80080FF49
:1039C000FCCF8091E30080688093E30083E01111D5
:1039D00001C082E08093AC0290CF8058823008F022
:1039E0008CCF8091AF029091B0028C3D23E0920782
:1039F00099F583E08A838AE289834FB7F894DE01E0
:103A0000139620E03EE051E2E32FF0E050935700A0
:103A1000E49120FF03C0E295EF703F5FEF708E2FBF
:103A200090E0EA30B8F0C7968D939D932F5F2431D4
:103A300059F74FBF8091E800877F8093E8006AE2E2
:103A400070E0CE01019646DC8091E8008B77809390
:103A5000E80053CFC096E8CF6091B1027091B202F6
:103A6000AE014F5F5F4F78DBBC01892B09F445CF76
:103A70009091E800977F9093E80089819A8189DC92
:103A8000E3CF803809F039CF8091E800877F8093B9
:103A9000E8008091A8028093F10024CF81112DCFFE
:103AA0009091AF02923008F028CF8091E800877F94
:103AB0008093E8009093A80200DD8091A8028823FB
:103AC00029F084E08093AC0249DA17CF8091E300BB
:103AD00087FDF7CF81E0F6CF0895CF938091AC02B8
:103AE000882391F0C091E900CF708091EC0080FDB7
:103AF0000DC080E0C82B1092E9008091E80083FDA2
:103B0000A6DECF70C093E900CF91089580E8F2CF90
:103B100097FB072E16F4009406D077FD08D048D006
:103B200007FC05D03EF4909581959F4F08957095C0
:103B300061957F4F0895EE0FFF1F0590F491E02DE2
:103B400009942F923F924F925F926F927F928F9241
:103B50009F92AF92BF92CF92DF92EF92FF920F931C
:103B60001F93CF93DF93CDB7DEB7CA1BDB0B0FB626
:103B7000F894DEBF0FBECDBF09942A8839884888E3
:103B80005F846E847D848C849B84AA84B984C88479
:103B9000DF80EE80FD800C811B81AA81B981CE0F70
:103BA000D11D0FB6F894DEBF0FBECDBFED01089555
:103BB000AA1BBB1B51E107C0AA1FBB1FA617B70753
:103BC00010F0A61BB70B881F991F5A95A9F780956F
:103BD0009095BC01CD010895FB01DC0104C08D91DD
:103BE0000190801921F441505040C8F7881B990B6F
:103BF0000895F999FECF92BD81BDF89A992780B5B5
:103C00000895A8E1B0E042E050E020C0262FF999E5
:103C1000FECF92BD81BDF89A019700B4021639F02B
:103C20001FBA20BD0FB6F894FA9AF99A0FBE0895FC
:103C30000396272FECDFEADF252FE9DF242FE7CFDC
:103C40000196272FE4DFE2CFDC01CB01FC01F999DB
:103C5000FECF06C0F2BDE1BDF89A319600B40D92D8
:0C3C600041505040B8F70895F894FFCF91
:103C6C002A024A02280850011E0A14010000010011
:103C7C001F16781773176E176917E200E900EA0030
:103C8C00B500B600B700CD008301CC008A019201CB
:103C9C0094012102230224022502260227022A0271
:103CAC00B300B4006F0070009F01CB019F02A00213
:103CBC00818283E200E900EA00B500B600B700CDCE
:103CCC00008301CC008A0192019401210223022479
:103CDC00022502260227022A02B300B4006F0070EC
:103CEC00009F01CB019F02A002818283946697C63C
:0A3CFC003435F4F5F6F731333236B3
:00000001FF
